:020000040000FA
:0400000069303A2801
:08000800A000030EA100831209
:1000100005191128831601178312B2308100B0012F
:100020002C2883160113831203140B190310A80D37
:10003000A90DAA0DAB0DAC0DAC16FF302C02031DA3
:100040002C28FA302B02031D2C2831152A08AF006A
:100050002908AE002808AD008B100B11210E83007B
:06006000A00E200E0900B5
:0C007400203084008001840A80300402E7
:10008000031C3C283B2283160C3085058701831214
:10009000850187010730990000309A0010308316DF
:1000A0008E008312603083168F0083120030831617
:1000B00091009F008312C830831681008312313073
:1000C0009000003083168C00831210308B00BC1B14
:1000D0006F2885196F286400851D6B28D7233C1C69
:1000E0007228382381018E018F010B118B100B10A8
:1000F0008C018B178A20311996201D22B30B88287A
:10010000031085190314B90DF030390203199E212B
:1001100049237A2864003210B00A301F9528AC01B8
:10012000AB01AA01A901A801B001080031110130F9
:10013000B70085144008013ECE000F08CF008B1396
:100140002030370783169B001C141A088312A40062
:100150001030370783169B001C141A088312A30063
:10016000A6000230A6060030370783169B001C1439
:100170001A088312A200A7000130A7068B17321CB1
:10018000C72822090339A200A309A409A509240844
:100190002F02031D982923082E02031D312922084E
:1001A0002D02031D982901303702031DDE283C195A
:1001B000DD283D18DE283D143E1458220230370257
:1001C000031DE9283C19E828BD18E928BD143E1490
:1001D000652203303702031DF4283C19F3283D192A
:1001E000F4283D153E14722204303702031DFF2807
:1001F0003C19FE28BD19FF28BD153E147F2205308D
:100200003702031D0A293C1909293D1A0A293D16FE
:100210003E148C2206303702031D15293C1914297F
:10022000BD1A1529BD163E14992207303702031D49
:1002300020293C191F293D1B20293D173E14A622C9
:1002400008303702031D2B293C192A29BD1B2B29F5
:10025000BD173E14B32209303702031D31293E1465
:10026000C02226082E02031D982927082D02031DEF
:10027000982901303702031D44293C1943293D1CAC
:1002800044293D103E14E72202303702031D4F2956
:100290003C194E29BD1C4F29BD103E14EB220330E2
:1002A0003702031D5A293C1959293D1D5A293D1170
:1002B0003E14EF2204303702031D65293C196429DE
:1002C000BD1D6529BD113E14F32205303702031D03
:1002D00070293C196F293D1E70293D123E14F722EA
:1002E00006303702031D7B293C197A29BD1E7B2964
:1002F000BD123E14FB2207303702031D86293C192C
:1003000085293D1F86293D133E14FF220830370200
:10031000031D91293C199029BD1F9129BD133E143D
:10032000032309303702031D97293E140723982918
:10033000B70A0A303702031808009F280130B600B8
:10034000B300B400B500B70085018701B1138A205E
:10035000B30BE429031085190314B90DF0303902E9
:1003600003190B2AB41F8510B40BE429013037029E
:1003700003190B230230370203190F23033037020E
:1003800003191323043037020319172305303702EA
:1003900003191B230630370203191F2307303702C6
:1003A00003192323083037020319272309303702A2
:1003B00003192B233708B6080319B6000319E229DD
:1003C0008514B6039630B400311DA7293111321CB3
:1003D000EE292D090339AD00AE09AF092F1CA7295D
:1003E0008E018F010C1CA7290C102E1EA7298B1320
:1003F00020303707BB002F08BA00262210303707FD
:10040000BB002E08BA00262200303707BB002D089B
:10041000BA0026228B178501870108303702203069
:10042000031985002A3003198700B70AB6010A307C
:100430003702031CA729382308003E1C08003E1081
:100440001030BB003D08BA00262208008B133A0882
:1004500083161C159A0083123B0883169B005530A7
:100460009D00AA309D009C1464009C18342A1C1125
:1004700083128B170800831600309B001C141A0887
:100480008312BC00831610309B001C141A088312C0
:100490003C18BD00831620309B001C141A088312E0
:1004A000C1000130C11BC100C1080319C10008000F
:1004B0003C19871640083C1D40034107D0000F0837
:1004C000D100BC1932233D1408003C19071640081E
:1004D0003C1D40034107D2000F08D300BC19322352
:1004E000BD1408003C19871540083C1D4003410716
:1004F000D4000F08D500BC1932233D1508003C1963
:10050000051640083C1D40034107D6000F08D700E0
:10051000BC193223BD1508003C19851640083C1D46
:1005200040034107D8000F08D900BC1932233D16FB
:1005300008003C19071540083C1D40034107DA003C
:100540000F08DB00BC193223BD1608003C198714C4
:1005500040083C1D40034107DC000F08DD00BC19CA
:1005600032233D1708003C19071440083C1D400386
:100570004107DE000F08DF00BC193223BD17080059
:10058000BC1908003C1DC82A303085043F30870460
:100590008E018F01C001D001D201D401D6010130FA
:1005A000D800DA00DC00DE004030D1008030D3001B
:1005B000C030D500FF30D7004030D9008030DB009C
:1005C000C030DD00FF30DF00FF30BD0008008712C3
:1005D0008E018F01080007128E018F01080087111C
:1005E0008E018F01080005128E018F01080085120F
:1005F0008E018F01080007118E018F0108008710FE
:100600008E018F01080007108E018F010800322330
:100610008E018F0108000708203A870008000708AC
:10062000103A870008000708083A87000800050804
:10063000103A850008000508203A850008000708E0
:10064000043A870008000708023A870008000708F4
:10065000013A870008000508303A850007083F3A4C
:1006600087000800CF308505C0308705BD01080030
:100670003D188716BD1807163D198715BD190516B3
:100680003D1A8516BD1A07153D1B8714BD1B07149F
:1006900008003C194D2B3D1C592B50084002031DEE
:1006A000592B51080F02031C592B3C1987123C1D72
:1006B00087163C195D2BBD1C692B52084002031D97
:1006C000692B53080F02031C692B3C1907123C1DB0
:1006D00007163C196D2B3D1D792B54084002031D54
:1006E000792B55080F02031C792B3C1987113C1DEF
:1006F00087153C197D2BBD1D892B56084002031D13
:10070000892B57080F02031C892B3C1905123C1D2D
:1007100005163C198D2B3D1E992B58084002031DD0
:10072000992B59080F02031C992B3C1985123C1D6B
:1007300085163C199D2BBD1EA92B5A084002031D8E
:10074000A92B5B080F02031CA92B3C1907113C1DA8
:1007500007153C19AD2B3D1FB92B5C084002031D4A
:10076000B92B5D080F02031CB92B3C1987103C1DE7
:1007700087143C19BD2BBD1FC92B5E084002031D09
:10078000C92B5F080F02031CC92B3C1907103C1D25
:1007900007144E084002031DD22B4F080F02031C02
:1007A000D22B85100C1C08000C10C00A0800B601E2
:1007B000B301B4013C1CDF2BBC01BC14EB2BBC1CF3
:1007C000E42BBC013C15EB2B3C1DE92BBC01BC15FB
:1007D000EB2BBC013C143C08B6006400EF2BF02B63
:1007E000F12BF22BF32BB41B8716B41F8712B30B1C
:1007F000ED2BB40BED2B0310B60CB608031DED2B3F
:0C0800000030BB003C08BA0026220800B3
:084000000800030006000600A1
:02400E00CC33B1
:10420000010078007A007C007E007B0079007F004E
:104210007D007A0078007E007C00FF00FF00FF0038
:104220000000F200F600FA00FE00F200F600FA00CC
:10423000FE00F200F600FA00FE00FF00FF00FF00A3
:10424000010005000500050005000900090009003E
:1042500009000D000D000D000D00FF00FF00FF0024
:10426000FF00FF00FF00FF00FF00FF00FF00FF0056
:10427000FF00FF00FF00FF00FF00FF00FF00FF0046
:10428000FF00FF00FF00FF00FF00FF00FF00FF0036
:10429000FF00FF00FF00FF00FF00FF00FF00FF0026
:1042A000FF00FF00FF00FF00FF00FF00FF00FF0016
:1042B000FF00FF00FF00FF00FF00FF00FF00FF0006
:1042C000FF00FF00FF00FF00FF00FF00FF00FF00F6
:1042D000FF00FF00FF00FF00FF00FF00FF00FF00E6
:1042E000FF00FF00FF00FF00FF00FF00FF00FF00D6
:1042F000FF00FF00FF00FF00FF00FF00FF00DD00E8
:00000001FF
